:100000000C94E6000C9472120C949F120C940E0146
:100010000C940E010C940E010C940E010C940E0124
:100020000C940E010C940E010C940E010C94D80C3F
:100030000C94AE100C940E010C940E010C940E0155
:100040000C94CC120C940E010C94FF130C940E0122
:100050000C940E010C940E010C940E010C940E01E4
:100060000C940E010C940E01746F6F206D616E790B
:10007000206F70656E2066696C6573006261642034
:10008000696E707574005941414B00594545454BA7
:100090000053616D706C65207261746520746F6FC0
:1000A0002068696768210000436F6D707265737323
:1000B000696F6E206E6F7420737570706F727465E7
:1000C00064006661696C656420746F2067657420E4
:1000D0006E657720636C7573746572002021212131
:1000E0002000203F3F3F2000204E6F74206120768B
:1000F000616C6964205741560020436F756C646ED3
:100100002774206F70656E2066696C65002E000A8A
:100110000D506C6179696E67200046696C657320CB
:10012000666F756E643A0046696C657320666F751C
:100130006E643A00436F756C646E2774206F70654F
:100140006E2064697200436F756C646E2774206F53
:1001500070656E2066696C65737973004E6F2070F0
:100160006172746974696F6E210043617264206901
:100170006E69742E206661696C656421000000243C
:10018000272A000025282B00002326290404040424
:100190000404040402020202020203030303030331
:1001A000010204081020408001020408102001020E
:1001B00004081020000000070002010000030406EC
:1001C0000000000000000000F810181211241FBEEB
:1001D000CFEFD4E0DEBFCDBF11E0A0E0B1E0EEE8AC
:1001E000F9E202C005900D92A232B107D9F714E0EE
:1001F000A2E2B1E001C01D92A836B107E1F711E01B
:10020000CCECD1E004C02297FE010E94C114C83C8E
:10021000D107C9F70E9411120C94C5140C94000068
:10022000FB01DC018D91019080190110D9F3990B2C
:100230000895FB01DC014150504030F08D91019058
:10024000801919F40020B9F7881B990B0895FB0158
:10025000DC014150504048F001900D920020C9F758
:1002600001C01D9241505040E0F708950895CB0120
:100270000E944D030895FC01848195810E9496049B
:100280000895EF92FF920F931F93CF93DF93EB01AB
:100290008A0179010BC0B801C7010E9410010097C3
:1002A00029F4CE010E94960481E006C0B701CE0178
:1002B0000E949F04882379F7DF91CF911F910F91BE
:1002C000FF90EF900895EF92FF920F931F93DF93AB
:1002D000CF93CDB7DEB768970FB6F894DEBF0FBEE9
:1002E000CDBF8C017E010894E11CF11C97010E9496
:1002F0004101882319F420E030E005C0B701C801AE
:100300000E9478089C01C90168960FB6F894DEBF78
:100310000FBECDBFCF91DF911F910F91FF90EF9056
:100320000895FC01AB0164817581828193810E94F3
:1003300063010895EF92FF920F931F93DF93CF9382
:10034000CDB7DEB768970FB6F894DEBF0FBECDBF4E
:100350008B017E010894E11CF11CB701FC01848132
:1003600095810E949F04882349F04CE050E0B7013A
:10037000C8010E942701F801148681E068960FB633
:10038000F894DEBF0FBECDBFCF91DF911F910F91CB
:10039000FF90EF900895EF92FF920F931F93DF93DA
:1003A000CF93CDB7DEB768970FB6F894DEBF0FBE18
:1003B000CDBF8C017E010894E11CF11CB701FC014A
:1003C000828193810E944205B701F8018281938165
:1003D0000E942907F8019583848320E0892B09F086
:1003E00021E0822F68960FB6F894DEBF0FBECDBF16
:1003F000CF91DF911F910F91FF90EF9008950F9390
:100400001F938C01FC01808191810E945305F801AA
:100410009383828320E0892B09F021E0822F1F91B2
:100420000F9108950F93CF93DF93EC0100E020E04C
:1004300030E040E050E069EF7AE08FE39AE00E941C
:10044000B70899838883892B69F40FEF20E030E0A7
:1004500040E050E069EF7AE08FE39AE00E94B7084D
:100460009983888320E088819981892B09F021E094
:10047000822FDF91CF910F9108950E94E90908958D
:10048000DC018C91853E39F1882329F1F901208125
:100490003181828193812817390799F444835583E8
:1004A000668377831B968C911B978F3011F080E2C7
:1004B00005C08C918295880F807E805E808780E069
:1004C00008951B968C918F3031F02F5F3F4F318311
:1004D000208381E0089581E008950F931F93CF93C7
:1004E000DF938C01FC018081853E09F48CC0882358
:1004F00009F489C0E9018C899D89AE89BF8900977B
:10050000A105B10521F44C8B5D8B6E8B7F8B209701
:1005100009F479C00115110509F475C0F80180814D
:10052000882309F470C083858F3011F481E06CC09A
:10053000A801D80180E090E0282F3C91303251F0A2
:10054000FE01E80FF91F30832F5F01961196883066
:10055000910591F78881853011F485EE8883F80143
:1005600080858032B1F0FE01E20FF11D8EE28083C2
:10057000822F8F5F2C5FFA019085903249F0FE0147
:10058000E80FF11D90838F5F4F5F5F4F821799F7E0
:10059000282FFE01E20FF11D1082F80183858D875F
:1005A000938D80E0228D30E0822B932B9F878E8766
:1005B000258D30E040E050E0542F432F322F22278A
:1005C000868D90E0A0E0B0E0DC0199278827282BF9
:1005D000392B4A2B5B2B848D90E0A0E0B0E0282BD8
:1005E000392B4A2B5B2B878D90E0A0E0B0E0B82F31
:1005F000AA2799278827282B392B4A2B5B2B288B56
:10060000398B4A8B5B8B80E0DF91CF911F910F91EB
:100610000895DF93CF9300D0CDB7DEB7DC0100970C
:10062000A1F16230710588F1ED91FC911197660F8F
:10063000771F80E090E016962D913D914D915C9151
:100640001997620F731F841F951F0190F081E02D91
:1006500022E030E0AE014F5F5F4F09958823A9F09B
:100660009A8180E0298130E0282B392B2115310532
:1006700071F08FEF273F380741F0C9014096079787
:1006800020F08FEF283F380710F020E030E0C9015C
:100690000F900F90CF91DF910895FC01009711F01A
:1006A0001182108208952F923F924F925F926F9223
:1006B0007F928F929F92AF92BF92CF92DF92EF92F2
:1006C000FF920F931F93DF93CF93CDB7DEB72C9795
:1006D0000FB6F894DEBF0FBECDBF3C0178876F83A5
:1006E0005A874987009709F402C1672B09F4FFC0B4
:1006F000452B09F4FCC0DC015A96AD90BD90CD901D
:10070000DC905D9752962D913D914D915C9155975E
:10071000E985FA85CF01A0E0B0E08A0D9B1DAC1DF4
:10072000BD1D281739074A075B0740F4B9016A194C
:100730007B097A876987672B09F4DCC0D301ED91C7
:10074000FC911197208931893A8329835E966D91B6
:100750007C915F977C876B87C901A0E0B0E08B83B9
:100760009C83AD83BE83672BE1F5F3010088F1899B
:10077000E02DFC87EB87EF2B39F4A114B104C10401
:10078000D10409F4B7C0B3C0A114B104C104D104A9
:1007900041F1860175012B803C804D805E80509434
:1007A000409430942094211C311C411C511C10C0D9
:1007B0006B857C85D3018D919C910E9409039C8758
:1007C0008B87892B09F493C0E20CF31C041D151DC3
:1007D0006B817C818D819E81E616F70608071907DB
:1007E00038F7C601B5012B813C814D815E810E94A5
:1007F00082142B0189849A84D301ED91FC91A98004
:10080000BA80A418B5088A149B0408F45401C08067
:10081000D180720100E010E086899789A08DB18DAA
:10082000E80EF91E0A1F1B1FEB85FC853297BF01DE
:1008300080E090E03296FC87EB872B813C814D81F4
:100840005E810E943C14E60EF71E081F191FD60198
:10085000ED91FC9195014F815885C801B70109952B
:10086000882361F18A189B08C501A0E0B0E0F3017C
:10087000228D338D448D558D280F391F4A1F5B1FE4
:10088000D3015A962D933D934D935C935D97C5018B
:10089000840D951DE981FA818E179F07B0F06B8555
:1008A0007C858D919C910E9409039C878B87892B65
:1008B00051F4D3015F961C921E925E9749855A852A
:1008C0004819590919C0442455242B853C85F30146
:1008D000378F268F8114910439F06F8178856A0DE6
:1008E0007B1D78876F8388CF49855A8505C04FEF78
:1008F0005FEF02C040E050E0CA012C960FB6F894BA
:10090000DEBF0FBECDBFCF91DF911F910F91FF9042
:10091000EF90DF90CF90BF90AF909F908F907F909F
:100920006F905F904F903F902F900895FC0100973B
:1009300011F480E00895138E128E81E008952F92B5
:100940003F924F925F926F927F928F929F92AF925F
:10095000BF92CF92DF92EF92FF920F931F93DF939C
:10096000CF93CDB7DEB7A9970FB6F894DEBF0FBE11
:10097000CDBF3C012B01009709F44AC061157105F8
:1009800009F446C0FC0180899189892B09F040C097
:10099000228D338DA081B1811097B9F1ED91FC9139
:1009A000119722803380AE014F5F5F4F89E0FA01DB
:1009B00011928A95E9F73C832B8352966D917D9134
:1009C0008D919C91559756960D911C915797061BAA
:1009D000170B6A0120E4E22E22E0F22E20E230E042
:1009E000AE01465F5F4FF1010995882371F08D805C
:1009F0009E80AF80B88481149104A104B10429F0D1
:100A000021C0F20180818823A9F5F301138E128E93
:100A100080E0A9960FB6F894DEBF0FBECDBFCF9190
:100A2000DF911F910F91FF90EF90DF90CF90BF90DB
:100A3000AF909F908F907F906F905F904F903F907E
:100A40002F90089588E1F20111928A95E9F70985BE
:100A500062019DE6E92E92E0F92E10E020E230E0FE
:100A6000AE01465F5F4FC501B401F10109958823CE
:100A700061F2C7CFF301828D938D0196938F828FA0
:100A800081E0C7CFFB01892B61F06115710549F049
:100A900088E1DB011D928A95E9F780E1858781E095
:100AA000089580E008952F923F924F925F926F9247
:100AB0007F928F929F92AF92BF92CF92DF92EF92EE
:100AC000FF920F931F93DF93CF93CDB7DEB7E097DD
:100AD0000FB6F894DEBF0FBECDBF6C01009709F4CE
:100AE00090C1ABC1EAE7F1E08AE1DF011D928A958E
:100AF000E9F7D0927B01C0927A01D60119962D9127
:100B00003D914D915C911C9719E0220F331F441FBA
:100B1000551F1A95D1F72AA33BA34CA35DA3CA0185
:100B2000B901655F7F4F8F4F9F4FED91FC9129E198
:100B300030E0AE014F5F5F4F0995882309F484C10F
:100B4000A9804A80BB81BEA30C81FD801E813F81AC
:100B5000588469847A849D8580E02C85E22FF0E0BA
:100B6000E82BF92B8E883F88288DE98C309709F483
:100B70006BC1432D50E060E070E0962F852F742FFD
:100B8000662769A77AA78BA79CA7822F90E0A0E091
:100B9000B0E0BC015527442789A59AA5ABA5BCA503
:100BA000842B952BA62BB72B482D50E060E070E0EE
:100BB000842B952BA62BB72B89A79AA7ABA7BCA7ED
:100BC0008E2D90E0A0E0B0E0782F662755274427CF
:100BD00089A59AA5ABA5BCA5842B952BA62BB72BD5
:100BE00089A79AA7ABA7BCA70097A105B10589F46F
:100BF000972D80E0662D70E0682B792B61157105CB
:100C000009F422C1CB01A0E0B0E089A79AA7ABA765
:100C1000BCA7942D80E02A2C3324282A392A952D2C
:100C200080E0A32FB0E0A82BB92BB8A7AFA39F2DCE
:100C300080E0202F30E0822B932B9C0140E050E09D
:100C40002A8F3B8F4C8F5D8FBF0180E090E0212F7A
:100C500030E040E050E00E943C146E8F7F8F88A30C
:100C600099A3E9A4FAA40BA51CA54A8D5B8D6C8DF4
:100C70007D8DE41AF50A060B170B6E8D7F8D88A10A
:100C800099A1E61AF70A080B190BC10101972FA1C8
:100C900038A5B5E0220F331FBA95E1F7820F931FF5
:100CA000B1010E945B1480E090E0E61AF70A080B9D
:100CB000190B7EA1272F30E040E050E0C801B701BA
:100CC0000E94821429013A01D301C201855F9F402D
:100CD000A040B0408050904FA040B04008F0B4C059
:100CE00086E0D60118968C93ACE78A2EA1E09A2E66
:100CF00088E1F40111928A95E9F75101CC24DD24B1
:100D000069A57AA58BA59CA5A60195010E943C1416
:100D100060937C0170937D0180937E0190937F01AD
:100D2000C601B5012A8D3B8D4C8D5D8D0E943C1412
:100D30007B018C012AA13BA14CA15DA1E20EF31E17
:100D4000041F151FE0928001F0928101009382013F
:100D50001093830142E050E060E070E0440E551EC5
:100D6000661E771E440C551C661C771C409284013D
:100D700050928501609286017092870130928901BC
:100D8000209288015EA1852F90E0BC01269EC001C3
:100D9000279E900D369E900D112490938B01809389
:100DA0008A016E8D7F8D88A199A1A60195010E946F
:100DB0003C146E0D7F1D801F911F60938C017093FA
:100DC0008D0180938E0190938F01AFA1B8A59D01F5
:100DD00040E050E0E5E0220F331F441F551FEA9525
:100DE000D1F7620F731F841F951F6093900170935A
:100DF000910180939201909393019401225030408D
:100E000002C020E030E0C901E0960FB6F894DEBFE2
:100E10000FBECDBFCF91DF911F910F91FF90EF904B
:100E2000DF90CF90BF90AF909F908F907F906F900A
:100E30005F904F903F902F90089580917A0190910C
:100E40007B01892BF1F64ECE10927B0110927A0134
:100E5000D8CFCF93DF939C01DB01009729F1611577
:100E6000710511F11D968C911D9784FF1DC0809115
:100E7000220190912301892B19F4E2E2F1E008C0EC
:100E800080913E0190913F01892B71F4EEE3F1E0F6
:100E9000EF01229688E10D9009928150E1F73183AC
:100EA0002083138E128E02C0E0E0F0E0CF01DF91CC
:100EB000CF9108952F923F924F925F926F927F92BF
:100EC0008F929F92AF92BF92CF92DF92EF92FF925A
:100ED0000F931F93DF93CF93CDB7DEB72A970FB64B
:100EE000F894DEBF0FBECDBF4C017C836B831A012B
:100EF000009709F4DEC0672B09F4DBC041155105EA
:100F000009F4D7C0DC015A96ED90FD900D911C912B
:100F10005D9780E09EEFAFEFBFEFE822F9220A2352
:100F20001B23D4015A96ED92FD920D931C935D976D
:100F300052962D913D914D915C9155972E153F05FF
:100F40004007510708F4B8C0C101A0E0B0E08E0D21
:100F50009F1DA01FB11F281739074A075B0728F4F8
:100F600019012E183F0809F4A7C0D401ED91FC9196
:100F70001197208931893A8329835E968D919C91BE
:100F80005F979A878987290166247724892BD9F569
:100F900050960D90BC91A02DBA87A987AB2B39F440
:100FA000E114F1040105110509F486C082C0E114C1
:100FB000F1040105110539F15701680188279927C6
:100FC000DC0184199509A609B7098D839E83AF8337
:100FD000B88714C069857A85D4018D919C910E944F
:100FE00009039A878987892B09F463C08D819E81C3
:100FF000AF81B885A80EB91ECA1EDB1EA414B504A5
:10100000C604D70438F7510191E0291692E0390659
:1010100018F0A12C82E0B82EC801B701A3019201FB
:101020000E9482147B0129813A81261B370B6501BE
:101030002A153B0508F4690100E010E0D401ED91A8
:10104000FC9186899789A08DB18DE80EF91E0A1F43
:101050001B1FE985FA853297BF0180E090E0329648
:10106000FA87E987A30192010E943C14E60EF71E5D
:10107000081F191F96014B815C81C801B7010E94AE
:101080004B0C892BC9F0960140E050E0F401828DB1
:10109000938DA48DB58D820F931FA41FB51F828FD2
:1010A000938FA48FB58F29853A85378F268FA50119
:1010B00005C04FEF5FEF02C040E050E0CA012A9642
:1010C0000FB6F894DEBF0FBECDBFCF91DF911F9159
:1010D0000F91FF90EF90DF90CF90BF90AF909F90D7
:1010E0008F907F906F905F904F903F902F900895DA
:1010F000CF93DF939C01FB01009731F061157105DF
:1011000019F0858584FF2CC060E08CE790E003C077
:1011100060E088E690E00E94B40C20E030E0C90175
:10112000DF91CF910895CCE5D1E0DF0188E10D900A
:1011300009928150E1F730935B0120935A0110929C
:1011400074011092750110927601109277018685D4
:10115000978590937901809378012AE531E0DFCF7C
:1011600080915A0190915B01892B91F6DCCF8F928F
:101170009F92AF92BF92CF92DF92EF92FF920F9326
:10118000DF93CF93CDB7DEB760970FB6F894DEBF8D
:101190000FBECDBF7C016B015A014901009709F4D4
:1011A00093C06115710509F48FC004300CF08CC038
:1011B00007FD1DC0602F772767FD7095E4E0660F7F
:1011C000771FEA95E1F762547E4F882777FD809577
:1011D000982F20E130E0AE014F5F5F4FF701099596
:1011E000882309F471C08D81882309F46DC0809132
:1011F0009C01882309F068C07CC08D8180939C018C
:101200002A8530E040E050E0542F432F322F222730
:101210008B8590E0A0E0B0E0DC0199278827282B9F
:10122000392B4A2B5B2B898590E0A0E0B0E0282B7E
:10123000392B4A2B5B2B8C8590E0A0E0B0E0B82FD7
:10124000AA2799278827282B392B4A2B5B2B2093F9
:101250009D0130939E0140939F015093A0012E85E4
:1012600030E040E050E0542F432F322F22278F856B
:1012700090E0A0E0B0E0DC0199278827282B392BEB
:101280004A2B5B2B8D8590E0A0E0B0E0282B392B1A
:101290004A2B5B2B888990E0A0E0B0E0B82FAA270A
:1012A00099278827282B392B4A2B5B2B2093A101C8
:1012B0003093A2014093A3015093A40103C08FEF88
:1012C00080939C019F0102C020E030E0C90160963C
:1012D0000FB6F894DEBF0FBECDBFCF91DF910F9157
:1012E000FF90EF90DF90CF90BF90AF909F908F9046
:1012F0000895E4E9F1E081E1DF011D928A95E9F7C3
:10130000F0929501E0929401D0929701C0929601DB
:10131000B0929901A092980190929B0180929A01BB
:1013200007FF6BCFCCCF282F8FEF8EBD0DB407FEFC
:10133000FDCF8DB58F778DBD8EB5822F80648EBD2C
:101340000DB407FEFDCF8DB58F778DBD872F992703
:10135000AA27BB278EBD0DB407FEFDCF8DB58F77B5
:101360008DBDCB01AA27BB278EBD0DB407FEFDCFD7
:101370008DB58F778DBDBB27A72F962F852F8EBD5F
:101380000DB407FEFDCF8DB58F778DBD4EBD0DB46D
:1013900007FEFDCF8DB58F778DBD222311F08FEF26
:1013A00001C085E98EBD0DB407FEFDCF8DB58F77E9
:1013B0008DBD90E02FEF2EBD0DB407FEFDCF8DB596
:1013C0008F778DBD8EB58F3F19F49F5F9A3099F757
:1013D0000895CF93DF93239A259A229A24982A9AE4
:1013E00083E58CBD8DB58E7F8DBD20E030E09FEF15
:1013F0009EBD0DB407FEFDCF8DB58F778DBD8EB52B
:101400002F5F3F4F2A30310599F72A98C0E0D0E08E
:1014100040E050E060E070E080E00E94930981309D
:1014200031F081E0CF3FD807E1F02196F1CFC0E065
:10143000D0E040E050E060E070E081E00E9493097D
:1014400080FF06C08FE7CF3FD80759F02196F1CF34
:1014500040E052E060E070E080E10E949309882360
:1014600019F02A9A80E008C02A9A8CB58C7F8CBD2E
:101470008DB581608DBD81E0DF91CF9108958F9210
:101480009F92AF92BF92DF92EF92FF920F931F93C2
:10149000CF93DF937B018C015A01E901DD24DA94BB
:1014A000812C42E0942E5EC02A98B801A7014070BA
:1014B0005E7F81E10E949309882319F02A9A80E0D7
:1014C00055C0DEBC0DB407FEFDCF8DB58F778DBD49
:1014D0008EB58E3FB1F7A7015170B401641B750B37
:1014E000C617D70708F4BE01FB01E40FF51F20E083
:1014F00030E0DEBC0DB407FEFDCF8DB58F778DBD1E
:101500008EB52417350730F02E173F0718F4D50194
:101510008D935D012F5F3F4FB2E020303B0749F7CD
:10152000DEBC0DB407FEFDCF8DB58F778DBD8EB5BA
:10153000DEBC0DB407FEFDCF8DB58F778DBD8EB5AA
:101540002A9ADEBC0DB407FEFDCF8DB58F778DBD19
:101550008EB5C61BD70BCB01A0E0B0E0E80EF91E9C
:101560000A1F1B1F209709F09FCF81E0DF91CF91C9
:101570001F910F91FF90EF90DF90BF90AF909F90E1
:101580008F90089520911A0130911B019FEF0AC09E
:101590009EBD0DB407FEFDCF8DB58F778DBD8EB589
:1015A0002F5F3F4F82E02030380790F38FEF8EBDE2
:1015B0000DB407FEFDCF8DB58F778DBD8EB58FEF46
:1015C0008EBD0DB407FEFDCF8DB58F778DBD8EB569
:1015D0002A9A8FEF8EBD0DB407FEFDCF8DB58F77A4
:1015E0008DBD8EB58FEF9FEF90931B0180931A01F5
:1015F00008952F923F924F925F926F927F928F92B7
:101600009F92AF92BF92CF92DF92EF92FF920F9391
:101610001F93DF93CF93CDB7DEB72C970FB6F89417
:10162000DEBF0FBECDBF4B015C011A013C872B878B
:101630002801FE82ED82D886CF824115510509F43A
:10164000DAC02115310509F4D6C00217130708F4D2
:10165000D2C0EF2809F4CFC02A98309521953F4F8A
:101660003A87298784011170D501C40180709E7F5B
:1016700089839A83AB83BC83AC01BD0181E10E9465
:101680009309882311F02A9AB6C09FEF9EBD0DB42E
:1016900007FEFDCF8DB58F778DBD8EB58E3FA9F737
:1016A00020E030E00BC0AFEFAEBD0DB407FEFDCFC4
:1016B0008DB58F778DBD8EB52F5F3F4F20173107CA
:1016C00090F3E12C52E0F52EE01AF10A3701EB8598
:1016D000FC856E1A7F0A6201CE1ADF0A00E012E072
:1016E0000E191F092B853C85E216F30648F14216B8
:1016F000530630F1F10120E030E00CC08FEF8EBDD9
:101700000DB407FEFDCF8DB58F778DBD8EB581935E
:101710002F5F3F4FAB85BC852A173B0778F3A801A5
:1017200060E070E0480D591D6A1D7B1D2F813885D2
:10173000C101ED81FE810995882321F491E026C045
:1017400090E024C02B853C85E21AF30A421A530A22
:1017500061147104A9F389859A85680E791EC80EF3
:10176000D91E020F131FC9018C0D9D1D892B09F075
:10177000B9CFE6CFAFEFAEBD0DB407FEFDCF8DB54F
:101780008F778DBD8EB50894E108F108E114F1045E
:1017900089F7BFEFBEBD0DB407FEFDCF8DB58F77C6
:1017A0008DBD8EB5EFEFEEBD0DB407FEFDCF8DB54F
:1017B0008F778DBD8EB52B853C854216530678F00C
:1017C000992369F489809A80AB80BC8080E092E0A4
:1017D000A0E0B0E0880E991EAA1EBB1E43CF2A9A35
:1017E0008FEF8EBD0DB407FEFDCF8DB58F778DBD0C
:1017F0008EB581E001C080E02C960FB6F894DEBF74
:101800000FBECDBFCF91DF911F910F91FF90EF9051
:10181000DF90CF90BF90AF909F908F907F906F9010
:101820005F904F903F902F900895FC0120911A01F6
:1018300030911B014FEF2F3F340731F460E086E811
:1018400090E00E94B40CFFCFCB01820F931F815018
:10185000924020F060E072E0621B730B20E030E009
:101860004FEF14C04EBD0DB407FEFDCF8DB58F7781
:101870008DBD8EB5819380911A0190911B010196C7
:1018800090931B0180931A012F5F3F4F2617370754
:1018900048F3CB010895CF92DF92EF92FF920F931E
:1018A0001F93CF93DF937B018C016A0180911A0112
:1018B00090911B018F5F9F4F31F060E08BE890E0CB
:1018C0000E94B40CFFCFE90182E02130380710F00C
:1018D000C0E0D2E02A9880E09EEFAFEFBFEFE822B1
:1018E000F9220A231B23B801A70181E10E94930971
:1018F000882321F02A9AC0E0D0E02CC09FEF9EBD43
:101900000DB407FEFDCF8DB58F778DBD8EB58E3FA3
:10191000B1F710921B0110921A012FEF14C02EBDC7
:101920000DB407FEFDCF8DB58F778DBD8EB5D60179
:101930008D936D0180911A0190911B0101969093F6
:101940001B0180931A0180911A0190911B018C1741
:101950009D0728F3CE01DF91CF911F910F91FF904A
:10196000EF90DF90CF9008950F931F93CF93DF9365
:10197000EC01062F10E005C082ED93E00E942812D2
:101980001F5FFE01E10FF11D64916623A9F700239B
:1019900051F06AE082ED93E00E9430126DE082ED3A
:1019A00093E00E943012DF91CF911F910F91089523
:1019B0001F920F920FB60F9211242F933F934F93C4
:1019C0008F939F93AF93BF93EF93FF93E091A50104
:1019D000F091A601309709F4A8C02091AB03309193
:1019E000AC038091AD039091AE032817390709F03D
:1019F00047C08091B0038823B9F18091A7039091EB
:101A0000A80327EA32E041E0873A940749F430938B
:101A1000A8032093A7039093AA038093A9030AC065
:101A200087EA91E09093A8038093A7033093AA03D9
:101A30002093A9038091A7039091A8039093AC03EE
:101A40008093AB0380509F4F9093AE038093AD0380
:101A50001092B0038091AF03882391F480916F00BE
:101A6000846080936F000CC081899289A389B489B6
:101A70000196A11DB11D818B928BA38BB48B55C098
:101A80005A985C985B9A5B985C9A5B9A5B985B9AB5
:101A90005B985B9A5B988781803119F5E091AB0385
:101AA000F091AC038181805890E087FF02C05C9A7E
:101AB00001C05C985B9A5B989F5F983011F0880F2B
:101AC000F4CF908180E097FF02C05C9A01C05C98DF
:101AD0005B9A5B988F5F843011F0990FF4CF329648
:101AE0001DC08830F9F4E091AB03F091AC03908114
:101AF00080E097FF02C05C9A01C05C985B9A5B989B
:101B00008F5F883011F0990FF4CF5B9A5B985B9AE6
:101B10005B985B9A5B985B9A5B983196F093AC0309
:101B2000E093AB035A9A5D985D9AFF91EF91BF9154
:101B3000AF919F918F914F913F912F910F900FBE39
:101B40000F901F9018950895CF93DF93EC0180912B
:101B50006F008D7F80936F008D89882319F00E941C
:101B6000C20A1D8AE091A501F091A601108A109287
:101B7000A6011092A501DF91CF910895CF92DF9237
:101B8000EF92FF920F931F93DF93CF93CDB7DEB702
:101B900028970FB6F894DEBF0FBECDBF8C016B0146
:101BA00044E050E07E010894E11CF11CB701C6013D
:101BB0000E945303049709F0F0C044E050E060E055
:101BC00071E0C7010E941901009709F0E6C0F5C055
:101BD00044E050E065E071E0CE0105960E941901F5
:101BE000009709F0DAC0F2C044E050E06AE071E02A
:101BF000C7010E941901009709F0CFC0F0C0542F0F
:101C0000432F322F22278081280F311D411D511D66
:101C10003197EC17FD0799F7F80124873587468738
:101C20005787203131054105510509F0B6C048E01C
:101C300050E0BE016F5F7F4FC6010E9453030897BB
:101C400009F0ABC08A8190E0A0E0B0E0BA2FA92FE4
:101C5000982F88272981820F911DA11DB11D019701
:101C6000A105B10521F061E088EA90E084C08C8193
:101C700090E0A0E0B0E02227382F492F5A2F8B8127
:101C8000280F311D411D511D2330310541055105DE
:101C900008F083C0F8012083FE013896BE016C5F16
:101CA0007F4F542F432F322F22278081280F311D41
:101CB000411D511D3197E617F70799F7F801218368
:101CC00032834383548348E050E0BE016F5F7F4F0F
:101CD000C6010E945303089709F05FC08E8190E00F
:101CE000A0E0B0E0BA2FA92F982F88272D81820F6E
:101CF000911DA11DB11DF80196838583888590E013
:101D0000A0E0B0E02227382F492F5A2F8F81280FCB
:101D1000311D411D511D213131054105510508F08D
:101D20003CC0278381819281A381B4818332F6E50F
:101D30009F07F0E0AF07F0E0BF0718F0293040F050
:101D40000CC081589E43A040B04050F0293040F074
:101D5000FF24F8018081823020F0FF24F39401C039
:101D6000FF2461E087EA90E00E94B40CFF2031F08C
:101D700061E081E990E00E94B40C0FC0F801108688
:101D8000118612861386D78AC68A118A128A138A06
:101D9000148A108A158A81E001C080E028960FB667
:101DA000F894DEBF0FBECDBFCF91DF911F910F9191
:101DB000FF90EF90DF90CF90089548E050E0B7019A
:101DC000C6010E945303089741F702CF44E050E058
:101DD000B701C6010E9453030497F9F605CFF80135
:101DE000148615861686178644E050E0B701C601B2
:101DF0000E945303049789F6F801248535854685AA
:101E00005785FE013496FBCEAF92BF92CF92DF9200
:101E1000EF92FF920F931F93DF93CF9300D000D0E8
:101E20000F92CDB7DEB76C015B01F42EE52EFC01FD
:101E300080859185A285B3850097A105B105D1F56F
:101E400044E050E08E010F5F1F4FB80186899789EB
:101E50000E945303049709F0F5C01D8244E050E04E
:101E6000B801D60156968D919C9157970E945303C5
:101E7000049709F0E7C0F6011086118612861386D2
:101E8000FE01349620E030E040E050E0542F432F34
:101E9000322F22278081280F311D411D511D31977E
:101EA000EC17FD0799F7D60118962D933D934D93A6
:101EB0005C931B978F2D9E2D9C017901B2E0213000
:101EC0003B0718F0E12C72E0F72EF60120853185F2
:101ED00042855385C701A0E0B0E0281739074A07BB
:101EE0005B0708F47901D6015696ED91FC9157975E
:101EF000828D938DA48DB58D9170A070B070009778
:101F0000A105B105D1F4D60155968C918823A9F489
:101F1000A701B501CF010E945A078C018E159F05BC
:101F200041F060E082EE90E00E94B40C0E94C20A90
:101F30008BC081E0F601858B73C0D60155968C91DC
:101F4000882309F463C0B701C5010E94150C5C0128
:101F50008E159F0539F060E08CED90E00E94B40C86
:101F60000E94C20AD6015696ED91FC915797C50181
:101F7000A0E0B0E0228D338D448D558D820F931FEC
:101F8000A41FB51F828F938FA48FB58F9170A070FF
:101F9000B0700097A105B10509F041C00E94C20AC6
:101FA000F601158A06891789D801ED90FC901197E2
:101FB000F7012089318940E050E05A966D917D917A
:101FC0008D919C915D970E94821461157105810528
:101FD000910529F5D8015E966D917C915F97C701B7
:101FE0000E940903F801978F868F892BC1F4D601CF
:101FF0005696ED91FC915797178E168E61E082EC04
:1020000090E00E94B40C0FEF1FEF1EC0A701B501B6
:10201000CF010E9453038E159F05A1F401C07501E5
:10202000970140E050E0F60180859185A285B38557
:10203000821B930BA40BB50B80879187A287B38774
:10204000870102C000E010E0C8010F900F900F90D0
:102050000F900F90CF91DF911F910F91FF90EF9014
:10206000DF90CF90BF90AF900895CF92DF92EF9224
:10207000FF920F931F93CF93DF93EC01C980DA8017
:10208000EB80FC809093A6018093A50107EA11E004
:102090001093AC030093AB0342E050E0B8010E9400
:1020A000040F892B09F451C08091AB039091AC03CC
:1020B00002969093AE038093AD03EE89FF89828DE3
:1020C00040E051E0481B5109B8016E5F7F4F80919D
:1020D000A5019091A6010E94040F9C010097A9F10F
:1020E0008091AD039091AE03820F931F9093AE0346
:1020F0008093AD0340E051E067EA72E08091A50172
:102100009091A6010E94040F81E08093B003888B18
:102110001092800089E08093810060E074E284EF97
:1021200090E0A70196010E948214309389002093C9
:10213000880081E090E090938B0080938A008091EA
:102140006F00826080936F007894DF91CF911F9130
:102150000F91FF90EF90DF90CF9008951F920F9214
:102160000FB60F9211242F933F934F935F936F936A
:102170007F938F939F93AF93BF93EF93FF93809140
:102180006F008B7F80936F008091B0038823F9F4F8
:1021900081E08093AF0378946091A9037091AA03C2
:1021A00040E051E08091A5019091A6010E94040FAA
:1021B000892B31F48091A5019091A6010E94A40D74
:1021C000F8941092AF0381E08093B0037894FF916C
:1021D000EF91BF91AF919F918F917F916F915F919F
:1021E0004F913F912F910F900FBE0F901F90189518
:1021F00081EB93E00E94360189EB93E00E94A30DEE
:102200000895BC0181EB93E00E949101BC01909381
:10221000B8038093B703009721F461E089EF90E061
:1022200009C089EB93E00E94BE0D882331F461E080
:1022300088EE90E00E94B40C089589EB93E00E9430
:10224000351008950E9401110BC060E08DE091E00F
:102250000E94B40C64E670E080E090E00E943C13C1
:102260008091C903882389F76091B7037091B803FF
:1022700081EB93E00E9437010895EF92FF921F9344
:10228000DF93CF93CDB7DEB72F970FB6F894DEBFAD
:102290000FBECDBF81EB93E00E943B0110E07E01B9
:1022A0000894E11CF11C0BC0B70181EB93E00E9484
:1022B0009A01882319F41092D1031FC01F5F8091E7
:1022C000D10390E0212F30E0821793076CF760E094
:1022D0008FE091E00E94B40CB70182ED93E00E9480
:1022E000381281EB93E00E943B01C7010E9422114A
:1022F0008091D1038F5F8093D1032F960FB6F8940E
:10230000DEBF0FBECDBFCF91DF911F91FF90EF9049
:1023100008950F931F93DF93CF93CDB7DEB72D971B
:102320000FB6F894DEBF0FBECDBF81EB93E00E94E5
:102330003B0161E08AE191E00E94B40C8E010F5FE5
:102340001F4FB80181EB93E00E949A01882379F432
:1023500081EB93E00E943B012D960FB6F894DEBF0F
:102360000FBECDBFCF91DF911F910F910895B8019E
:1023700082ED93E00E946712E4CF40E855E260E00E
:1023800070E082ED93E00E9423126FE071E082ED35
:1023900093E00E94671261E082E00E94A01361E076
:1023A00083E00E94A01361E084E00E94A01361E03A
:1023B00085E00E94A01361E089E00E94A01381EBF8
:1023C00093E00E943D02882321F461E08AE691E0D7
:1023D0001DC081EB93E00E941202882321F461E08A
:1023E0008CE591E013C081EB93E00E94FF0188230C
:1023F00021F461E086E491E009C081EB93E00E9462
:10240000CB01882331F461E084E391E00E94B40CB5
:10241000089561E087E291E00E94B40C0E94891166
:1024200008950E9466130E94BD110E943D11FDCFC8
:1024300080E291E09093D3038093D2030895862F96
:102440000E94F7130895CB01BA010E94BE130895AC
:10245000DC01ED91FC910190F081E02D099508954A
:10246000DC01ED91FC910190F081E02D099508953A
:102470000F931F93CF93DF938C01EB0109C021963B
:10248000D801ED91FC910190F081E02DC8010995F2
:1024900068816623A1F7DF91CF911F910F91089575
:1024A0000F931F938C01DC01ED91FC910190F08161
:1024B000E02D6DE00995D801ED91FC910190F0813E
:1024C000E02D6AE0C80109951F910F9108950F93BF
:1024D0001F938C010E943812C8010E9450121F9154
:1024E0000F9108951F920F920FB60F9211242F9300
:1024F0003F934F935F936F937F938F939F93AF938C
:10250000BF93EF93FF938091D4039091D503892BD0
:1025100029F0E091D403F091D5030995FF91EF9153
:10252000BF91AF919F918F917F916F915F914F91EB
:102530003F912F910F900FBE0F901F9018951F92F3
:102540000F920FB60F9211242F933F934F935F93E7
:102550006F937F938F939F93AF93BF93EF93FF936B
:102560008091D6039091D703892B29F0E091D6036F
:10257000F091D7030995FF91EF91BF91AF919F9192
:102580008F917F916F915F914F913F912F910F901C
:102590000FBE0F901F9018951F920F920FB60F92BB
:1025A00011242F938F939F93AF93BF938091D80360
:1025B0009091D903A091DA03B091DB030196A11D9C
:1025C000B11D8093D8039093D903A093DA03B093FD
:1025D000DB038091DC039091DD03A091DE03B091D9
:1025E000DF038050904CAF4FBF4F8093DC0390933C
:1025F000DD03A093DE03B093DF0327C08091DC03EB
:102600009091DD03A091DE03B091DF0380589E43DB
:10261000A040B0408093DC039093DD03A093DE03E1
:10262000B093DF038091E0039091E103A091E20376
:10263000B091E3030196A11DB11D8093E003909337
:10264000E103A093E203B093E3038091DC03909154
:10265000DD03A091DE03B091DF0381589E43A040CB
:10266000B04060F6BF91AF919F918F912F910F90E5
:102670000FBE0F901F901895EF92FF920F931F932C
:102680007B018C018FB7F8944091E0035091E103F6
:102690006091E2037091E3038FBF2FB7F8948091AC
:1026A000E0039091E103A091E203B091E3032FBF17
:1026B000841B950BA60BB70BE816F9060A071B0738
:1026C00060F71F910F91FF90EF900895789484B573
:1026D000826084BD84B5816084BD85B5826085BD1E
:1026E00085B5816085BDEEE6F0E080818160808304
:1026F000E1E8F0E080818260808380818160808376
:10270000E0E8F0E0808181608083E1EBF0E08081AF
:1027100084608083E0EBF0E0808181608083EAE781
:10272000F0E080818460808380818260808380810A
:10273000816080838081806880831092C1000895C9
:10274000282F30E0C90180569E4FFC0194912457F8
:102750003E4FF9018491882381F0E82FF0E0E3589F
:10276000FE4FE491F0E0662329F48081909589235F
:10277000808308958081892B80830895EF92FF9252
:102780000F931F937B018C0122E030E040E050E08A
:102790000E94A414205C3D4B404F5F4FCA01B90119
:1027A000A80197010E94A414C901DA010197A109A7
:1027B000B109292F3A2F4B2F552747FD5A950196DE
:1027C000A11DB11D2093C50081508093C400E1EC90
:1027D000F0E0808180618083808188608083808157
:1027E000806880831F910F91FF90EF900895982F3C
:1027F0008091C00085FFFCCF9093C60008951F9282
:102800000F920FB60F9211242F933F934F935F9324
:102810006F937F938F939F93AF93BF93EF93FF93A8
:102820004091C600E091E403F091E503CF010196E9
:1028300060E870E00E946F149C018091E603909123
:10284000E7032817390739F0E851FC4F40833093EC
:10285000E5032093E403FF91EF91BF91AF919F9126
:102860008F917F916F915F914F913F912F910F9039
:102870000FBE0F901F901895629FD001739FF001BB
:10288000829FE00DF11D649FE00DF11D929FF00D00
:10289000839FF00D749FF00D659FF00D9927729F37
:1028A000B00DE11DF91F639FB00DE11DF91FBD01C2
:1028B000CF0111240895AA1BBB1B51E107C0AA1F19
:1028C000BB1FA617B70710F0A61BB70B881F991FD1
:1028D0005A95A9F780959095BC01CD01089597FB75
:1028E000092E07260AD077FD04D0E5DF06D00020A8
:1028F0001AF4709561957F4F0895F6F7909581953C
:102900009F4F0895A1E21A2EAA1BBB1BFD010DC00B
:10291000AA1FBB1FEE1FFF1FA217B307E407F5078F
:1029200020F0A21BB30BE40BF50B661F771F881F6B
:10293000991F1A9469F760957095809590959B0101
:10294000AC01BD01CF01089597FB092E05260ED0DD
:1029500057FD04D0D7DF0AD0001C38F450954095BD
:10296000309521953F4F4F4F5F4F0895F6F7909563
:102970008095709561957F4F8F4F9F4F0895EE0F13
:0E298000FF1F0590F491E02D0994F894FFCF0D
:10298E0052494646005741564500666D7420005721
:10299E0061766520746573742100FFFF00000000EE
:0229AE001F12F6
:00000001FF
